:020000040100F9
:10000000382A00205D010001690E0001CD0D0001BC
:1000100000000000000000000000000000000000E0
:100020000000000000000000000000005512000168
:1000300000000000000000001B0100015912000137
:100040006F0100016F0100016F0100016F010001EC
:100050006F0100016F0100016F0100016F010001DC
:100060006F0100016F0100016F0100016F010001CC
:100070006F0100016F0100016F0100016F010001BC
:100080006F0100016F0100016F0100016F010001AC
:100090006F0100016F0100016F0100016F0100019C
:1000A0006F0100016F0100016F0100016F0100018C
:1000B000BD1300016F0100016F0100016F0100011C
:1000C0000348854600F09EFA00480047512300018E
:1000D000382A002040BA7047C0BA70470138FDD1B5
:1000E00070470000084B19680868203080F30988C1
:1000F000022080F31488BFF36F8F3FBCAE4608BC6C
:1001000004BC62B61847000004000020EFF3108022
:1001100072B6704780F310887047EFF309800E4B7A
:100120001A6820381060F0C044464D4656465F4677
:10013000F0C008B572B602F0DBFE62B60CBC116806
:1001400008681030F0C8A046A946B246BB4680F306
:1001500009882038F0C81847040000200448804768
:1001600004480047FEE7FEE7FEE7FEE7FEE7FEE79E
:100170008D120001C100000130B50B460146002080
:100180002022012409E00D46D5409D4205D31D469D
:100190009540491B2546954040191546521E002D95
:1001A000F1DC30BD03460B439B0703D009E008C9CF
:1001B000121F08C0042AFAD203E00B780370401C17
:1001C000491C521EF9D27047D2B201E00270401CA5
:1001D000491EFBD270470022F6E710B513460A46C7
:1001E00004461946FFF7F0FF204610BD421C017877
:1001F000401C0029FBD1801A704710B5002200E096
:10020000521C835C8C5CA34201D1002BF8D1D8B284
:10021000E1B2401A10BDF0B51FB40646002082B00E
:1002200005464024019100901BE0019922460F46AB
:10023000304600F009FA049A059B801A994110D3C0
:1002400010461946224600F0EFF9361A8F41019701
:10025000224601200021009F00F0E6F938184D41A8
:1002600000902046641E0028DFDC019B0098294690
:10027000324607B0F0BD0000F0B5074608465840CA
:1002800087B0C00F049048000E4659004008490846
:10029000BC1A884105D2384631461E4617460B46E1
:1002A00002465800400810434CD0300D03904005E2
:1002B0005900400D490D0590401A0290402872DA0D
:1002C00018030121000B09050843019004980092CE
:1002D000002805D0019952420020884100920190E7
:1002E000029840210A1A0199009800F09DF90546EC
:1002F0000C466B4607CB00F0B8F9C0197141039A60
:100300000E0D0023D71756401A467A40164344D0A4
:10031000049A002A2DD0029A012A039A15DC1205AC
:10032000C01A914101263605001C7141D20F059E6D
:10033000D2070093019202962A46234600F0B5F9AF
:1003400007B0F0BD38463146FAE71605224A0F4697
:10035000B218C01AB74101210905001C4F4100180D
:100360007F41114618187941E20F10436D1964411D
:1003700013E0E2076D0815436408C2071443039AAB
:1003800001261205C01A91413605001C7141CE07A5
:10039000400830434908C01851412A46234600F01E
:1003A00077F9CDE7FFE7049801224000C117121A40
:1003B00000238B4104983146C417381AA141EEE757
:1003C00030B40124E407634030BC55E730B4012465
:1003D000E407614030BC4FE70000E0FFF0B51FB418
:1003E00088B00B990998002448400999C00F49002A
:1003F00049080991C0070B990090490049080B91E1
:1004000009990898A64608431CD00B990A980843F6
:1004100018D0099801244000420D4800410D099868
:1004200024050003000B204309900B980003000BE8
:1004300020430B9050181C4940180022019014468C
:10044000104605E0002001460DB0F0BD032801DA9A
:10045000034600E003239C46C11A0AAE0AE05F008F
:1004600008ADED5B4F00F75B7D430027AA187C4188
:10047000491C5B1E6145F2DD410004AB5A52210468
:10048000120C0A43240C401C0828DFDB0198029060
:100490000099704601910090059B049A079906986F
:1004A00000F003F9D0E700000DFCFFFFF0B50C46AB
:1004B0005C4085B0E40FE40703944C000026640818
:1004C00059009446490802460296224321D06246CA
:1004D0000A431ED06200570D4A000E032303550D38
:1004E000012402462C492405781B1B0B360B4018AF
:1004F00023432643614600901C46501AB44103D35F
:100500000098401C009002E0921800985B4100287F
:1005100003DA0020014605B0F0BD002001210905E5
:100520000746864611E064461D46141BB54106D3B6
:100530006546521BB341744607430C43A646CD079C
:1005400040084908284392185B4105460D43EAD10B
:100550001046184313D06046194650407140084376
:1005600006D06046101AB34106D20122002306E0ED
:1005700000220123DB0702E00122D243531000983E
:1005800074460105381C6141029C039D00196941B4
:1005900000F07EF8BFE70000FD0300004A000903F9
:1005A0000123090B1B0519430A4B10B5520D9A4242
:1005B00002DA0020014610BD064B34339A4203DCB8
:1005C0009A1A00F041F810BD034BD21800F02CF835
:1005D00010BD0000FF030000CDFBFFFF10B5002998
:1005E00004DB0124E40740428C412146002B04DB5C
:1005F0001C460123DB075242A341994200D190429D
:1006000010BD0000064C0125064E05E0E36807CC4E
:100610002B430C3C98471034B442F7D3FFF754FDFA
:10062000083D0001283D000110B5202A04DB0146E9
:10063000203A9140002010BD914020239C1A03468F
:10064000E3401943904010BD10B5202A04DB084652
:10065000203AD040002110BD0B46D340D04020248A
:10066000A21A91400843194610BD10B5202A06DB96
:10067000CB170846203A1041C1170B4306E00B4642
:100680001341D0402024A21A91400843194610BDBE
:1006900010B5002B08DA0024401C614192185B4120
:1006A0001A4301D14008400010BDF0B51FB482B01C
:1006B00005460C0003D0084600F090FF02E000F071
:1006C0008DFF20300246009021462846FFF7ACFF00
:1006D000049B059A04460F4618431143084314D05F
:1006E000184610431BD0009840210A1A1846059955
:1006F000FFF7AAFF05460E46009A05990498FFF7F2
:1007000093FF084305D0012004E02046394607B096
:10071000F0BD0020C11705430E432C433743009919
:100720000E986305401A7905E40A00220C43FD0A7D
:100730000A3002D500200146E9E701051019694198
:100740000C9C0D9D00196941FFF7A2FFDFE7000037
:100750001CB5002003210346FF22013200910190C5
:1007600002A1034802F038FF1CBD0000434C4900C1
:100770000D0800011CB5002208210A2002F023FC0C
:100780001049086000200221034680220091019058
:100790000DA10F4802F020FF002002210346802215
:1007A000009101900BA10D4802F016FF00200321DB
:1007B0000346FF2201320091019009A10A4802F08C
:1007C0000BFF1CBD640000204C45443100000000BC
:1007D000D10D00014C454432000000001D0E000107
:1007E0005052494E54000000F50F000101480078B6
:1007F0007047000068000020002801D0012100E0BF
:100800000021014A117070476800002008B50024DB
:10081000002531A001F04AFD00BF0021C943684610
:1008200001F004FC002800D1F7E7002D07D028468E
:10083000002569460978814200D1EEE700BF68468D
:1008400000780D2803D0684600780A2819D1684638
:1008500000780D2801D10A2000E00D20054601F0A6
:1008600033FC29A001F022FD002028490855084644
:1008700001F09EFC22A001F019FD01F037FC0024DC
:1008800028E068460078082803D0684600787F286A
:1008900007D1002C1EDD601E84B21DA001F006FDF4
:1008A00018E068460078202814DB684600787F2826
:1008B00010DA3F2C0BDA684602782046611C8CB2B5
:1008C00012490A540121684601F024FC02E011A0FB
:1008D00001F0ECFCA1E700000D0A434C49207265D1
:1008E0006164792E2054797065202768656C7027C3
:1008F00020666F7220636F6D6D616E64732E0D0ADA
:100900006E33323E200000000D0A0000F42100206A
:10091000082008000700000070B505460E460AA032
:1009200001F0C4FC00240BE00C206043094BC0180C
:1009300042680C206043195807A001F09DFC641C1C
:10094000042CF1D370BD0000636F6D6D616E647334
:100950003A0D0A002C3C00012020252D387320255B
:10096000730D0A00F8B507460C46032F03DA25A0DD
:1009700001F09CFCF8BD60680078312806D1606801
:100980004078002802D1284D01260EE060680078EA
:10099000322806D160684078002802D1234D4026D5
:1009A00003E018A001F082FCE4E721A1A068FFF7B2
:1009B00024FC002804D13146284601F0B9FA19E098
:1009C0001CA1A068FFF719FC002804D13146284675
:1009D00001F0A6FA0EE018A1A068FFF70EFC0028AF
:1009E00004D13146284601F0ABFA03E005A001F03E
:1009F0005DFCBFE712A0A268616801F03DFC00BF8A
:100A0000B8E7000075736167653A206C6564203C47
:100A1000317C323E203C6F6E7C6F66667C746F6703
:100A2000676C653E0D0A0000000C014000080140A3
:100A30006F6E00006F666600746F67676C6500001C
:100A40006C656420257320257320646F6E650D0A24
:100A50000000000070B505460C46022D0CDAFFF7C9
:100A6000C5FE002801D017A000E017A006463146B9
:100A700016A001F001FC70BD12A16068FFF7BDFB7C
:100A8000002803D10120FFF7B7FE0CE00EA160683B
:100A9000FFF7B3FB002802D1FFF7AEFE03E00EA084
:100AA00001F004FCE7E7FFF7A1FE002801D005A054
:100AB00000E005A0064631460DA001F0DDFB00BFB9
:100AC000D9E700006F6E00006F6666006C6F6720EC
:100AD00069732025730D0A0075736167653A206C90
:100AE0006F67205B6F6E7C6F66665D0D0A000000AD
:100AF0006C6F672073657420746F2025730D0A0076
:100B000070B504460D4604A001F0D0FB0F48016803
:100B10000FA001F0B1FB70BD4E333257423033317C
:100B2000204672656552544F53202B205541525434
:100B300028444D4129202B204C4544202B20434C58
:100B4000492064656D6F0D0A000000000000002060
:100B500053797374656D436F7265436C6F636B207B
:100B60003D20256C7520487A0D0A000048607047CA
:100B70000168254A114001600021016041608160E7
:100B8000C1602249884208D12049083949680F22AA
:100B900011431E4A083A516035E01C49143188421D
:100BA00008D11A4908394968F0221143174A083A0E
:100BB000516028E015492831884209D11349083984
:100BC00049680F2212021143104A083A51601AE094
:100BD0000E493C31884209D10C49083949680F2235
:100BE00012031143094A083A51600CE00749503199
:100BF000884208D10549083949680F221204114377
:100C0000024A083A51607047FEFF000008000240A7
:100C1000002904D0026801231A43026003E002683D
:100C2000014B1A4002607047FEFF000010B50246FB
:100C3000002000230B681C461440002C01D001202A
:100C400000E0002010BD000010B5002202680D4B2E
:100C50001A400C6A8B6823430C6923434C69234375
:100C60008C692343CC6923434C6A23438C6A234316
:100C70001A430260CB6843600B6883604B68C360B3
:100C800010BD00000F80FFFF10B5002B01D01061D8
:100C900001E00024146110BD70B503460A4600212E
:100CA0000024002076E001268E40156835402C4651
:100CB000002C6ED05568022D02D05568122D20D11F
:100CC00008250D40002D0ED0586A4D07EE0E0F2559
:100CD000B5400646AE4330464E07F60E5569B54060
:100CE000284358620DE0186A4D07EE0E0F25B540F7
:100CF0000646AE4330464E07F60E5569B5402843CA
:100D000018625568012D08D05568112D05D0556819
:100D1000022D02D05568122D0BD1586801258D4047
:100D20000646AE4330461579ED06ED0F8D4028435B
:100D3000586018684E000325B5400646AE4330465D
:100D40001579AD07AD0F4E00B54028431860D8683F
:100D50004E000325B5400646AE4330464E0095682A
:100D6000B5402843D860986801258D400646AE43BB
:100D70003046D5688D4028439860D86A4E000125DA
:100D8000B5400646AE4330464E001569B54028438F
:100D9000D862491C1568CD40002D84D170BD00007B
:100DA000054901600F2141610021416081600121FD
:100DB000C160002101617047FF3F00008162704700
:100DC0008161704742694A404261704700BFFEE757
:100DD0001CB50F4903C90191009000BF01210D48C6
:100DE00001F0AEF8FFF702FD00280BD001206946A4
:100DF00008700198401C019000231A4606480068BC
:100E000002F04AF9FF20F53001F092FFE6E700001A
:100E10001C3C0001000C0140640000201CB50F497F
:100E200003C90191009000BF40210D4801F088F8EE
:100E3000FFF7DCFC00280BD00220694608700198FF
:100E4000401C019000231A460648006802F024F96D
:100E50007D20C00001F06CFFE6E70000243C0001AB
:100E600000080140640000207047000010B50446EF
:100E700061780020205600F01BF8A078002809D0E7
:100E800000202056C206D20E01219140074A11606F
:100E900000BF0AE000202056C206D20E0121914078
:100EA000024A8032116000BF00BF10BD00E100E0C7
:100EB00010B5002819DA1A4A03071B0F083B9B08D4
:100EC0009B00D2588307DC0EFF23A3409A438B0775
:100ED0001B0E8407E40EA3401A43114B0407240F92
:100EE000083CA408A4001A5118E00E4A03231B0270
:100EF000D21883089B00D2588307DC0EFF23A3403F
:100F00009A438B071B0E8407E40EA3401A43054B3C
:100F1000032424021B198408A4001A5110BD0000E8
:100F20001CED00E000E100E0F7B5D4B004460E4649
:100F300000205390052052900025002700BFEFF3BA
:100F400010800090FF21453101A8FFF744F901F01E
:100F500013FE05462448854218D10120000384422F
:100F600002D1002053902AE001204003844202D1A4
:100F70004011539023E003200003844203D1012059
:100F8000400253901BE0529857B0F0BD174885427D
:100F900013D101200003844201D153900FE00120BE
:100FA0004003844201D1539009E0032000038442AE
:100FB00001D1539003E05298E6E75298E4E705AF79
:100FC0000137FF2241320A4901A8FFF7EBF801205F
:100FD00000F02AFB3146569A5398B8475290009831
:100FE00000F022FB5298CFE7C44013008560130045
:100FF000383A00011CB500BF0022D24369460848B8
:10100000006802F054F90128F6D101F05DF8684655
:10101000017804A0019A00F0BBFA01F067F8EBE751
:10102000640000204C4544257520746F67676C652B
:10103000642C20636F756E74203D20256C750A004A
:10104000002905D0054A52690243044B5A6104E065
:10105000024A52698243014B5A61704700100240B4
:10106000002905D0054A92690243044B9A6104E0C5
:10107000024A92698243014B9A6170470010024014
:1010800010B500210022214B5B680424234019463F
:10109000002902D0042906D102E01D4B036005E0BF
:1010A0001C4B036002E01A4B036000BF00BF174BEC
:1010B0005B683024234019460909174B5A5C0368C2
:1010C000D3404360114B5B68072424022340194638
:1010D000090A124B5A5C4368D34083600B4B5B6830
:1010E000E40023401946C90A0C4B5A5C4368D340BC
:1010F000C360064BDB6A10242340002B02D0084B50
:10110000036102E07D23DB03036110BD0010024098
:101110000090D0030048E801183C0001103C000199
:1011200000093D00F1B58AB0002009907D20C00083
:1011300008900125AD020027002007907F2006902F
:1011400040240026002005900390200102900020FA
:1011500001903E490A98884206D83D4800686102DD
:1011600088433B49086006E0394800680121C9030B
:101170000843374908607D21C9000A98FEF7FCFF43
:101180007D21C9000090FEF7F7FF450100BF304800
:1011900000687F21090288430190200201990843D9
:1011A0002B4908600520FEF799FF10E00120FEF7AB
:1011B00095FF2748406B02210840002800D007E037
:1011C0000598411C05910899884200D900E0EDE797
:1011D00000BF1F48C06B86B2AE4201D9771B00E04A
:1011E000AF1B0298874203D2E0B20390B8B20290DC
:1011F000AE4201D3069400E0079406990798401880
:10120000C005000E04900498A04200D103E0049CA5
:1012100009988742BBD800BF0D4800687F210902AA
:101220008843019003980002019908430849086027
:101230000846406840084000486000BF04484068D5
:10124000042108400028F9D10BB0F0BD0090D00374
:10125000001002407047000010B5FEF757FF04462B
:1012600002F0FAF9002803D0012000070249486083
:101270002046FEF74FFF10BD00ED00E00148024997
:10128000086070470090D0030000002010B53E4871
:10129000C0690121090708433B49C8618120000654
:1012A0003A4908633A4848613A4808623A4800684F
:1012B000032189038843384908603421374800F006
:1012C00073F836480069401C002803D03348006991
:1012D000002817D12C4840680121090408432A49F5
:1012E000486008464068072109028843264948604B
:1012F0000846406809150843234948602848FFF715
:1013000011FF3FE0214880694409640123480078C7
:10131000C006C00E04431D4884611B4800680121BB
:10132000C903884318490860084600687F210902FC
:1013300088430446194800690002204312490860A6
:10134000084640680121090408430F4948600846DF
:1013500040680721090288430B49486008464068F5
:1013600009150843084948600846006A0D490840C5
:10137000054908620846006A0849C9680902084325
:101380000149086210BD00000010024000700040DA
:101390000F0800001800020000100140700000203B
:1013A0000090D003FF00F8FF70B504460D462A46B2
:1013B000214601200003FFF7B7FD70BD10B500F016
:1013C00059FE10BDF8B503460024002600960025FE
:1013D0000020104EB14200D100BF18460E06740F17
:1013E000CE06F60E00960127009EB7403D46012C22
:1013F00001D10C3004E0022C01D1103000E0143097
:10140000002A03D006682E43066002E00668AE4359
:101410000660F8BD6A090000002905D08289012311
:101420005B031A43828103E08289024B1A40828166
:1014300070470000FFDF0000002A03D0838A0B43BF
:10144000838202E0838A8B438382704702460020B6
:1014500001235B02994200D100BF13880B40002B8F
:1014600001D0012000E000207047000070B5024666
:101470000024002300250020124EB14200D100BFFD
:101480000E06750FCB06DB0E01269E403346012D5E
:1014900002D19689334006E0022D02D1168A3340EC
:1014A00001E0968A33400C120126A6403446168885
:1014B0003440002B03D0002C01D0012000E000209C
:1014C00070BD00006A090000F0B589B005460E46FF
:1014D00000240020089000BF00BF0027B08900282A
:1014E00000D000BF2F462C8A20480440F0880443D7
:1014F0002C82AC891E480440B08831890843718928
:1015000008430443AC81AC8A1A480440B0890443C0
:10151000AC8201A8FFF7B4FD1748874202D10498B6
:10152000089001E003980890326891001923089A06
:101530005A431046FEF720FE079064210798FEF7F5
:101540001BFE04012109642041430798411A0691BA
:1015500006990901084632306421FEF70DFE0007A6
:10156000000F04432C8109B0F0BD0000FFCF000044
:10157000F3E90000FFFC00000038014001468888C4
:10158000C005C00D7047CA05D20D828070470000AB
:101590000FB410B503A9044B044A029800F002F9F5
:1015A00010BC08BC04B01847C52200016C00002024
:1015B0007CB51546024600201C4600290BD0491E6A
:1015C00000920191044B6A462146284600F0EAF851
:1015D000009A002111707CBDDD1E00012021020C4B
:1015E00001D010211046020A01D010460839020924
:1015F00001D01046091F820801D01046891E4208FA
:1016000001D0881E7047081A704702E008C8121FF0
:1016100008C1002AFAD170477047002001E001C1DB
:10162000121F002AFBD1704780F31088704700001A
:10163000F0B51FB486B00998089A030D0021024343
:1016400014D05148514A18185043051411980128D4
:1016500010981AD0281A401C00264D4F4D4900966C
:1016600001910490002812DA444211E011980124FB
:1016700049A3012801D11098C1430698119A8460AA
:101680000360C26041600BB0F0BD4042E4E7044635
:10169000210500203F4A001C51410391029012E0B5
:1016A000E00707D032463B4601990098FEF796FEC8
:1016B0000191009032463B4610461946FEF78EFED9
:1016C00006460F466410002CEAD10498039B0028BC
:1016D000029A0999089806DAFEF780FE019B009AA3
:1016E000FEF77CFE05E0FEF7E1FE019B009AFEF7A7
:1016F000DDFE04460E460022284BFEF76FFF03D89E
:101700000020C043014607E00022254B2046314619
:10171000FEF7B2FDFEF742FF102409E0002C0ADBC1
:101720000A220023FEF777FD079B30321A55641E0C
:1017300002460A43F2D11122641C079B121B1C199A
:10174000119B012B03D0012308430ED10AE008436B
:1017500004D0112010900020119077E71098151AEE
:101760006D1E0BE01098824202DD00236D1C03E029
:10177000824201DA00236D1E002BEED006981199EB
:101780008260C16030C07EE701FCFFFF104D0000A9
:10179000000014400000F03F300000000000F04363
:1017A0000000E03FFFB597B00646002518E2252867
:1017B00077D100242746FD49049400E00443761CB9
:1017C00032780120203A90400842F7D130782A2818
:1017D0000ED00222307801463039092916D80499F2
:1017E0000A235943303940181443761C0490F1E71A
:1017F000189802C804911890002904DA01204003C7
:1018000004434842049002200443761C30782E287A
:1018100014D1042004437078761C2A2809D1189822
:10182000761C80C8189009E00A214F43303FC71941
:10183000761C3078014630390929F5D930786C2882
:1018400010D006DC4C281AD068280ED06A2817D190
:1018500004E0742813D07A2812D110E0012040054A
:1018600004430CE00121090501E0032109050C43B3
:101870007178814203D1012000052418761C761C62
:101880003078119066280BD013DC58287DD009DC05
:1018900000287BD04528F6D04628F4D047281AD116
:1018A000A5E118E0632835D0642870D0652812D1EE
:1018B0009DE170286CD008DC6728F1D069287BD0C6
:1018C0006E280DD06F2806D1BAE073282ED0752867
:1018D00071D0782859D01A9A199990476D1C7EE1D9
:1018E0006002400F022809D003280DD00428189860
:1018F00001680DD00D60001D189070E11898EA176E
:1019000001680D604A60F6E7189801680D80F2E7FB
:101910000D70F0E718986A4601781172001D189052
:101920000020507202A80090012005E0189802C81B
:10193000189000200091C04361070DD5002101E0FF
:101940000199491C0191B94212DA8142F8DB009AEF
:10195000515C0029F4D10BE0002101E00199491C00
:1019600001918142FADB019A0099895C0029F5D145
:10197000019904981A9B471A21463846199A00F093
:1019800097FA0199401945180BE04FE02CE113E05C
:101990004EE0009800990078491C00911A9A199914
:1019A00090470198401E0190401CF2D121463846D4
:1019B0001A9B199A10E137E00A200021009001914A
:1019C0006002410F022907D0189A01CA1892C21763
:1019D0009446032908D00AE01898C01DC108C90020
:1019E00005C91891944607E000B2C217944604292D
:1019F00002D140B2C1178C4600226146944506DAF6
:101A00000A460021404291418C462D2102E02105E9
:101A100004D52B216A461173012103E0E10701D0AF
:101A20002021F7E7029155E00A200AE0102008E0A3
:101A3000102000900021042004430191082703E0B6
:101A400008200021019100906002410F022907D077
:101A5000189A01CA189200229446032908D008E077
:101A60001898C01DC108C90005C91891944603E023
:101A700080B2042900D1C0B200210291210729D5EA
:101A80001199702906D0009A1021019B4A401A43EF
:101A900005D00EE040216A461173012108E061463D
:101AA000014306D030216A46117311995173022106
:101AB0000291009A0821019B4A401A430AD16146CB
:101AC000014301D1610705D530216A461173012117
:101AD0007F1E02911199582904D035A10E910DA9AC
:101AE0000D910DE037A1F9E76146019B009AFEF7E1
:101AF00092FB0E9B8C469B5C0D9A521E0D921370AE
:101B000061460143F0D10D9805A9081A20300190D3
:101B1000600703D501200004844300E001270198F9
:101B2000874201DD381A00E0002001990090411839
:101B3000029809180498401A0490E00306D421463C
:101B40001A9B199A049800F0B3F94519002706E08A
:101B500003A81A9AC05D199990476D1C7F1C0298C2
:101B60008742F5DBE0030CD521461A9B199A0498AD
:101B700000F09EF9451904E01A9A3020199990470F
:101B80006D1C0099481E00900029F5DC08E00D98B6
:101B90000D990078491C0D911A9A199990476D1C5E
:101BA0000199481E01900029F1DC63E10928010038
:101BB00030313233343536373839616263646566C3
:101BC0000000000030313233343536373839414285
:101BD000434445460000000000F05AF94519761CC0
:101BE0003078002800D0E2E528461BB0F0BD600741
:101BF00000D406271898C01DC108C90048680A68A3
:101C00000831C30FDB071891190001D09CA108E02F
:101C1000210501D59BA104E0E10701D09AA100E0D4
:101C20009AA1430011985B08109165280CD006DC3E
:101C3000452809D046281DD0472841D141E06628D3
:101C400018D067283CD13CE00021112F01DB112086
:101C500000E0781C0191009008A911A8FFF7E8FCAA
:101C6000139905910021119A15927F1C12980197E2
:101C7000009150E00120C00703900120019008A9C5
:101C8000009711A8FFF7D4FC139A1499059200222B
:101C9000119B009212981593059A0192002901D088
:101CA000104602E0791C40180190381A01D50198BD
:101CB00004E04042401E0090781C0190C01B02903E
:101CC00043E0012F00DA01270021112F01DD11204F
:101CD00000E038460191009008A911A8FFF7A8FC80
:101CE00013990591119A002112981592009101976C
:101CF00021070CD40599B94201DB019900E001915B
:101D0000012904DD159A491E515C302906D0B842DC
:101D100001DA011D05DA0121029115E00199491E40
:101D2000EDE7002805DC0099411800910199091A96
:101D300003E0019A411C914200DD01910099401A93
:101D4000401C02900120C0070390200706D402998E
:101D50000198814202DB0020C043029000206946C6
:101D6000C87707AF012103980337C907884224D0F9
:101D7000022011902B201290039800280CDA404288
:101D800003902D20129007E00A210398FEF7F4F942
:101D900030317F1E039039701199481E119000292F
:101DA000F2DC03980028EFD1791E12980870307881
:101DB000202108404530BF1E387006A8C01BC01D3A
:101DC000039010980078002800D001200199411854
:101DD0000298C0170918039809180498401A401E61
:101DE0000490E00306D421461A9B199A049800F047
:101DF0005FF8451910980078002803D01A9A1999AD
:101E000090476D1CE00324D521461A9B199A04982B
:101E100000F04EF845191CE00098002807DB0099F7
:101E20000598884203DD1598405C199901E01999DD
:101E300030201A9A904700986D1C401C0090029820
:101E4000401E0290002804D11A9A2E20199990471A
:101E50006D1C0199481E01900029DDDC05E03878F1
:101E60001A9A7F1C199990476D1C0399481E03907C
:101E70000029F4DC21461A9B199A0498ACE600006C
:101E80002D0000002B0000002000000000000000DA
:101E9000F8B5044600251E461746880404D405E01C
:101EA00039462020B0476D1C641EF9D52846F8BD80
:101EB000FFB50446002581B01E46C80301D5302772
:101EC00000E02027880404D505E038460399B04790
:101ED0006D1C641EF9D5284605B0F0BD4A68002A7D
:101EE00006D00A68531C0B6010704868401E48609A
:101EF0007047000010B50121074800F003FA4021A7
:101F0000064800F0FFF90121034800F009F84021DC
:101F1000024800F005F810BD000C01400008014027
:101F200070B504460D4629462046FEF747FF70BDB2
:101F300070B504460D4629462046FEF741FF70BDA8
:101F400070B504460D4629462046FEF73BFF70BD9E
:101F500000B58BB001210820FFF782F8012188032A
:101F6000FFF77EF805A8FEF71BFF40200590022032
:101F7000069004200A9005A92648FEF78DFE8020D1
:101F8000059004200A9005A92248FEF785FEE1206D
:101F900040020190002168460181418181810182D6
:101FA0000C21C18101A91C48FFF78EFA01210846C6
:101FB000FFF746F81948FEF7DBFD0123174A1749DA
:101FC00008390220FEF760FE012280211248FFF747
:101FD00033FA00220121402000F0F5FF104908608B
:101FE000012000F0E1FF0F49086001220E490A4874
:101FF000FFF7E8F91C2168460170032141700121B7
:102000008170FEF733FF01210348FFF705FA0BB09B
:1020100000BD0000000C01400038014008000240F3
:102020005C000020600000202505000070B505461A
:102030000C460F480068002800D170BD601C0028C5
:1020400001D1401E07E07D21C900614308467D2182
:10205000C900FEF791F80646324629460448006852
:1020600001F025F9012800D1E7E70020E5E70000AD
:102070005C0000201CB5002001900F490F48FFF7BD
:10208000F5F9002817D00D48FFF778FAC0B2009094
:102090000B480068002806D0002301AA69460848BA
:1020A000006801F0A6F80198002803D0012000077D
:1020B0000449486000BF1CBD2505000000380140F0
:1020C0005C00002000ED00E010B507480068002823
:1020D00008D001F0AFFA022804D1C11E02480068FE
:1020E00001F081F910BD00006000002010B5084823
:1020F000006800280AD001F09DFA022806D10023CA
:102100001A4619460248006800F0C6FF10BD0000DC
:102110006000002030B58BB004460D46002C01D085
:10212000002D01D10BB030BD00211F48FEF770FD1E
:102130001D4908390220FEF719FD1C480090019442
:10214000102002900395002004908020059000202C
:1021500006900790089003200003099000200A9041
:1021600069461148FEF770FD01210F48FEF750FD4A
:1021700000BF0D4908390220FEF758FD0028F8D0AD
:1021800000210948FEF744FD074908390220FEF7FF
:10219000EDFC00BF40210548001FFFF757F900285C
:1021A000F8D000BFBEE7000008000240043801403C
:1021B000F0B589B0074600263C4621E000E0641CEB
:1021C00020782028FBD020780928F8D02078002813
:1021D00000D11AE03046761C800001A90C5000E0C6
:1021E000641C2078002805D02078202802D0207890
:1021F0000928F5D12078002802D000202070641C26
:102200002078002801D0082ED8DB00BF002E01D195
:1022100009B0F0BD002512E00C226A430C4B99581E
:102220000198FDF7EAFF002808D10C20684308490F
:10223000401801A9826830469047E9E76D1C042DDB
:10224000EAD304A0019900F017F800BFE0E700000E
:102250002C3C0001756E6B6E6F776E20636F6D6D39
:10226000616E643A2025732028747279202768658E
:102270006C7027290D0A00000FB408B503A8009060
:1022800060210948009B029AFFF792F90020009014
:10229000002105484030C177403800F007F801B010
:1022A00008BC04B0184700009421002070B5044613
:1022B0002046FDF79BFF85B229462046FFF72AFFFF
:1022C00070BD000070B504460D460A2C0AD10D21E0
:1022D0000B48FFF758F900BF80210948FFF7B6F80F
:1022E0000028F9D0E1B20648FFF74DF900BF802180
:1022F0000348FFF7ABF80028F9D0204670BD000076
:102300000038014030B587B004460D460E4884427F
:1023100004D101210420FEF7A3FE09E00B4884420A
:1023200004D101210820FEF79BFE01E007B030BD7B
:1023300001A8FEF735FD01950120029001A9204674
:10234000FEF7AAFC00BFF1E700080140000C0140C5
:10235000FEF794FFFFF7FCFD0BA0FFF719F915A09E
:10236000FFF716F91D4801681DA0FFF711F923A01A
:10237000FFF70EF9FFF7BEFDFEF7FCF9FEF7E8F9EF
:1023800000F078FD00BFFEE70A3D3D3D3D3D3D3D8F
:102390003D3D3D3D3D3D3D3D3D3D3D3D3D3D3D3D6D
:1023A0003D3D3D3D3D3D3D3D3D3D3D3D3D3D3D3D5D
:1023B0003D0A0000204E33325742303331204672FE
:1023C000656552544F53202B2055415254202B20E9
:1023D0004C45442064656D6F0A0000000000002039
:1023E0002053797374656D436F7265436C6F636BD3
:1023F000203D20256C7520487A0A00003D3D3D3D7A
:102400003D3D3D3D3D3D3D3D3D3D3D3D3D3D3D3DFC
:102410003D3D3D3D3D3D3D3D3D3D3D3D3D3D3D3DEC
:102420003D3D3D3D0A000000F8B505460E46174803
:10243000076817480068001D00F0C0FB681C0028F2
:1024400008D1002E06D012480168091D114800F07D
:10245000F4FB1AE07C190E4800684460BC4207D2C5
:102460000B480168091D0C48006800F0CBFB0CE02C
:1024700007480168091D0948006800F0C3FB0848C7
:102480000068844201D206480460F8BD18000020AC
:1024900004000020800100200C0000200800002023
:1024A0003400002010B5044600F0D4FB2248006838
:1024B000401C2149086021480068002808D11F48B5
:1024C00004600846006801280ED100F097F90BE07F
:1024D0001B480068002807D118480068C06AE16AF4
:1024E000884201D81548046016480068401C154908
:1024F00008600846006860641349E06A0968884219
:1025000002D91149E06A08601422E16A51430F4A76
:102510008818211D00F091FB00F0AAFB0848006814
:10252000002807D005480068C06AE16A884201D2E5
:1025300000F0F2FB10BD0000140000200400002099
:1025400020000020300000201C000020A4000020FB
:1025500010B516E000F07EFB0C48C068C468201D72
:1025600000F02CFB0A480068401E09490860094831
:102570000068401E0749086000F07AFB204600F022
:1025800061F8044800680028E4D110BD6C01002007
:10259000140000201000002070B504460D46206C89
:1025A00000280ED0216CE0684018E0606168E068A7
:1025B000884201D32068E0602846226CE168FDF77C
:1025C000F1FD70BDF8B504460F4615460020009099
:1025D000A66B206C002809D1206800282ED16068E5
:1025E00001F0D8F800900020606027E0002D0FD1A6
:1025F0003946226CA068FDF7D5FD216CA068401813
:10260000A0606168A068884218D32068A06015E0C7
:102610003946226CE068FDF7C5FD216CE068401A80
:10262000E0602168E068884203D2216C6068401A4B
:10263000E060022D02D1002E00D0761E701CA06337
:102640000098F8BD10B50446206B00F025FB20462D
:1026500000F022FB10BD01464A6A002A04D00A6B32
:1026600012680723981A00E00020704730B5012354
:102670005B0317484407640F002C05D0C01DC00839
:10268000C000134C041B1B1B0246124C226000248A
:10269000104D6C60D0180838C008C0000E4C206087
:1026A00000240D4D2D686C600B4D2D682C6011467B
:1026B000441A4C60084C24680C60084D4C682C602F
:1026C000074D4C682C600124E407064D2C6030BD9A
:1026D00094010020440000204C0000205400002001
:1026E000500000205800002000BFFFF731FF0348D2
:1026F00000680128F9D900F00FFBF6E7A4000020DC
:1027000010B50446002C09D0002060602060E06015
:1027100000231A461946204600F0BEFC10BDFFB546
:1027200081B006460D4617460A9C002D01D1246053
:1027300000E02760E66325640121204600F06BFC81
:102740004C210498085505B0F0BDFFB581B00F4687
:102750000A9E0C9C039A9100A522206BFDF734FD84
:10276000216B0398401E8000081800900098C00854
:10277000C000009000984007400F002801D10120C0
:1027800000E00020002802D172B600BFFEE700255D
:1027900008E0795D204634304155785D002800D14D
:1027A00002E06D1C102DF4D300BF00214320015521
:1027B000072E00D30626E662E66400202065201D71
:1027C00000F01DFA2046183000F019FA24610720A5
:1027D000801BA061646200206065002158200155C3
:1027E000049A0199009800F0B7F920600B9800282E
:1027F00001D00B98046005B0F0BD000010B50024B6
:1028000006E0142161430E4A881800F0EBF9641CBD
:10281000072CF6D30B4800F0E5F90B4800F0E2F97D
:102820000A4800F0DFF90A4800F0DCF9094800F036
:10283000D9F904480849086003480849086010BDF0
:10284000A400002030010020440100205801002095
:102850006C01002080010020080000200C000020F6
:1028600010B50146164800E0006803688B42FBD3B0
:10287000024643689B188B4204D143684C681B197D
:10288000436001460A464B689B180468A34211D175
:102890000C4C03682468A34208D04B680468646841
:1028A0001B194B6003681B680B6005E0054B1B6838
:1028B0000B6001E003680B60884200D0016010BD2E
:1028C000440000204C00002070B5054600F0C2F91D
:1028D000A86B002801D1012400E0002400F0C8F911
:1028E000204670BD70B5054600F0B4F9A86BE96BE1
:1028F000884201D1012400E0002400F0B9F920460B
:1029000070BD00000B4909680968002901D1012147
:1029100000E00021002904D00021C943064A1160CB
:1029200006E004490968C968C868034A416811603B
:1029300070470000080000203400002010B500207F
:102940000749086188617D21C90006480068FDF7D4
:1029500013FC401E024948610720086110BD0000B9
:1029600000E000E00000002007480068401C00284C
:1029700001D1012000E00020002802D172B600BF82
:10298000FEE772B600BFFEE74000002070B50446C7
:1029900000F060F94520055713E0606A002801D176
:1029A000012000E00020002808D12046243000F05B
:1029B00087FF002803D000F0E9F900E003E0681E7B
:1029C00045B2002DE9DC00BF0021C9434520015577
:1029D00000F04EF900F03EF94420055713E020695D
:1029E000002801D1012000E0002000280AD1204663
:1029F000103000F065FF002801D000F0C7F9681E14
:102A000045B200E001E0002DE9DC00BF0021C94330
:102A10004420015500F02CF970BD0000F8B50446C3
:102A20000020009000F05CFA3E480068002801D1C8
:102A3000FFF71CFE3C4800682040002861D1002CB4
:102A400015D008346007400F002810D06007400FF1
:102A50000821081A04196007400F002801D101203D
:102A600000E00020002802D172B600BFFEE7002C73
:102A700047D02E480068844243D82D4E3046056822
:102A800001E02E462D686868A04202D2286800281E
:102A9000F7D124480068854233D030680830009070
:102AA000286830606868001B102813D92F19780730
:102AB000400F002801D1012000E00020002802D1B1
:102AC00072B600BFFEE76868001B78606C6038462D
:102AD000FFF7C6FE154968680968081A13490860B7
:102AE0000846006813490968884203D20F48006805
:102AF000104908600C49686809680843686000204C
:102B0000286000F021FF00984007400F002801D105
:102B1000012000E00020002802D172B600BFFEE7CD
:102B20000098F8BD4C000020580000205000002004
:102B3000440000205400002006480068002806D009
:102B40000449096808465030096D491C0160014874
:102B50000068704704000020001F01231B0603606B
:102B6000001F0160001F034B03601438026020380F
:102B7000704700006929000170B5D2B0002400251B
:102B800000BFEFF310800646FF21453101A8FDF795
:102B900022FB01AC01349822074901A8FDF702FB92
:102BA0000120FEF741FDA04705463046FEF73CFDFB
:102BB000284652B070BD0000783B000101460A690A
:102BC0004B68886898608B6848685860506888428D
:102BD00001D188685060002008611068401E1060B4
:102BE000106870470146083141600021C943816087
:102BF00001460831C1600161002101607047002178
:102C00000161704710B502460B685C1C002C01D1B5
:102C1000106907E01046083000E040684468246806
:102C20009C42FAD944684C604C68A160886041605D
:102C30000A611468641C146010BD42684A6093689D
:102C40008B60936859609160086103685B1C036046
:102C50007047000072B605480068401C03490860D0
:102C6000BFF34F8FBFF36F8F70470000400000200D
:102C700008480068002802D172B600BFFEE7054888
:102C80000068401E0349086008460068002800D11B
:102C900062B670474000002070B506463546002EEB
:102CA00035D0083D2C461A4960680968084000285C
:102CB00001D0012000E00020002802D172B600BF40
:102CC000FEE72068002801D1012000E00020002854
:102CD00002D172B600BFFEE70D496068096808407E
:102CE000002814D02068002811D1094960680968BB
:102CF0008843606000F0F4F806496068096840188D
:102D0000044908602046FFF7ABFD00F01DFE70BDD2
:102D100058000020500000200120000703494860AF
:102D2000BFF34F8FBFF36F8F7047000000ED00E0DF
:102D300070B504460025002C14D00D48006800280A
:102D400001D1012000E00020002802D172B600BFAE
:102D5000FEE700F0C5F800212046FFF765FB00F014
:102D6000F3FD0546002D01D1FFF7D6FF70BD000031
:102D70003C0000200349096801600349096841607B
:102D8000704700002C00002018000020012001499D
:102D9000086070472800002070B504460D46002CDE
:102DA00002D172B600BFFEE705480168183120461F
:102DB000FFF728FF01212846FFF736FB70BD000012
:102DC00004000020FEB506460F4634460120009060
:102DD000002E48D0206D002802D172B600BFFEE759
:102DE000E06CB84201D23D4600E0E56CE06AA842E2
:102DF00039D0206D012836D11B480068844201D0AB
:102E0000012000E00020002802D172B600BFFEE7DA
:102E1000E06A0190E562A069C00FC007002802D1F6
:102E20000720401BA06161691422019850430F4A9A
:102E30008018814201D1012000E00020002812D03A
:102E4000201DFFF7BBFE0A49E06A0968884202D9E3
:102E50000749E06A08601422E16A5143034A88186E
:102E6000211DFFF7EAFEFEBD04000020A4000020A3
:102E70001C0000201CB5134800210B468022009145
:102E8000019011A1124800F0A7FB0446012C0DD1BE
:102E900072B60020C0430F49086001200E49086047
:102EA00000200E49086000F063F80AE0601C00286A
:102EB00001D0012000E00020002802D172B600BF3E
:102EC000FEE71CBD3800002049444C4500000000CE
:102ED000E926000134000020200000201800002016
:102EE00002480068401C0149086070473C0000200F
:102EF0001A480068002803D00120194908602CE016
:102F00000020174908601748016805E0002902D130
:102F100072B600BFFEE7491E14204843124A1058FB
:102F2000002801D1012000E000200028EED1142269
:102F30004A430D4BD018426852684260024608323C
:102F40004368934202D14268526842604268D26844
:102F5000064B1A600348016000BF70473C00002028
:102F6000280000201C000020A400002004000020F5
:102F700010B50B48006AFF2109040843084908629C
:102F80000846006AFF210906084305490862FFF761
:102F9000D5FC002003490860FDF7A4F8002010BD0F
:102FA00000ED00E040000020F8B5044601260027AF
:102FB00022460021012000F006F805462846FFF7CA
:102FC0009FFB2846F8BDF7B582B005460E46002D9A
:102FD00001D0012000E00020002802D172B600BF1D
:102FE000FEE7002E01D1002701E02F467743384647
:102FF0005030FFF713FD0446002C09D02046503016
:103000000190009431462846049B019AFFF787FB04
:10301000204605B0F0BD70B505460E462C46002C86
:1030200002D172B600BFFEE7FFF714FE216CE06B21
:1030300048432168401860600020A0632068A060B9
:10304000E06B401E216C484321684018E06000217D
:10305000C9434420015545200155002E10D1206957
:10306000002801D1012000E00020002810D12046D6
:10307000103000F025FC00280AD0FFF74DFE07E0D5
:1030800020461030FFF7AEFD20462430FFF7AAFDA2
:10309000FFF7EEFD012070BDFFB583B006461D466B
:1030A000002002903446002C02D172B600BFFEE729
:1030B0000498002802D1206C002801D1012000E0F2
:1030C0000020002802D172B600BFFEE7022D02D117
:1030D000E06B012801D1012000E00020002802D18E
:1030E00072B600BFFEE700F0A5FA002802D10598ED
:1030F000002801D1012000E00020002802D172B692
:1031000000BFFEE700BFFFF7A5FDA06BE16B8842A3
:1031100001D3022D1FD12A4620460499FFF752FA07
:103120000746606A002801D1012000E00020002845
:1031300008D12046243000F0C3FB002806D0FFF75A
:10314000EBFD03E0002F01D0FFF7E6FDFFF790FD58
:10315000012007B0F0BD0598002803D1FFF788FDD6
:103160000020F6E70298002804D16846FFF702FE27
:1031700001200290FFF77CFDFFF7B2FEFFF76AFD2A
:1031800044210857401C002802D100214420015549
:1031900045210857401C002802D100214520015537
:1031A000FFF766FD05A9684600F0DCF9002819D193
:1031B0002046FFF797FB00280ED0204610300599D7
:1031C000FFF7EAFD2046FFF7E1FB00F0BDFB00281A
:1031D00099D1FFF7A1FD96E72046FFF7D7FB00F056
:1031E000B3FB90E72046FFF7D1FB00F0ADFB0020DA
:1031F000AFE7FFB583B0064617461D463446002CA0
:1032000002D172B600BFFEE70498002802D1206CFC
:10321000002801D1012000E00020002802D172B670
:1032200000BFFEE7022D02D1E06B012801D1012091
:1032300000E00020002802D172B600BFFEE7FCF7D4
:1032400065FF0190A06BE16B884201D3022D26D16E
:103250004520015700912A4620460499FFF7B2F90C
:103260000098401C002812D1606A002801D101207A
:1032700000E0002000280FD12046243000F020FB81
:10328000002809D0002F07D00120386004E0009802
:10329000401C41B2452001550120029001E0002070
:1032A00002900198FCF736FF029807B0F0BDF7B521
:1032B00084B005460E46002003902C46002C02D117
:1032C00072B600BFFEE7002E02D1206C002801D1AB
:1032D000012000E00020002802D172B600BFFEE706
:1032E00000F0A8F9002802D10698002801D1012099
:1032F00000E00020002802D172B600BFFEE700BF48
:10330000FFF7A8FCA76B002F1AD031462046FFF725
:1033100043F9781EA0632069002801D1012000E054
:103320000020002807D12046103000F0C9FA0028FC
:1033300001D0FFF7F1FCFFF79BFC012007B0F0BDC7
:103340000698002803D1FFF793FC0020F6E70398C6
:10335000002804D101A8FFF70DFD01200390FFF71D
:1033600087FCFFF7BDFDFFF775FC44210857401CA3
:10337000002802D100214420015545210857401C56
:10338000002802D1002145200155FFF771FC06A954
:1033900001A800F0E7F8002819D12046FFF794FAB9
:1033A00000280ED0204624300699FFF7F5FC204671
:1033B000FFF7ECFA00F0C8FA0028A1D1FFF7ACFC47
:1033C0009EE72046FFF7E2FA00F0BEFA98E72046B3
:1033D000FFF7DCFA00F0B8FA2046FFF775FA00288C
:1033E0008ED00020AAE7F3B583B0054600200290F6
:1033F0002C460026002C02D172B600BFFEE7206CDE
:10340000002801D1012000E00020002802D172B67E
:1034100000BFFEE700F00EF9002802D10498002852
:1034200001D1012000E00020002802D172B600BFC7
:10343000FEE700BFFFF70EFCA76B002F1CD0781E25
:10344000A0632068002802D1FFF776FB6060206946
:10345000002801D1012000E00020002807D12046EB
:10346000103000F02DFA002801D0FFF755FCFFF7CF
:10347000FFFB012005B0F0BD049800280DD1002EFF
:1034800001D1012000E00020002802D172B600BF67
:10349000FEE7FFF7EDFB0020ECE70298002804D1DF
:1034A0006846FFF767FC01200290FFF7E1FBFFF79A
:1034B00017FDFFF7CFFB44210857401C002802D11D
:1034C00000214420015545210857401C002802D105
:1034D000002145200155FFF7CBFB04A9684600F009
:1034E00041F8002824D12046FFF7EEF9002819D032
:1034F0002068002807D1FFF7ADFB606800F08EF967
:103500000646FFF7B5FB204624300499FFF744FC3C
:103510002046FFF73BFA00F017FA00288AD1FFF7A0
:10352000FBFB87E72046FFF731FA00F00DFA81E751
:103530002046FFF72BFA00F007FA2046FFF7C4F900
:103540000028EED0002E0BD0FFF784FB2046FFF7BB
:1035500082F8074639466068FFF734FCFFF788FBBE
:10356000002087E770B505460C46002D02D172B6E3
:1035700000BFFEE7002C02D172B600BFFEE7FFF7E6
:1035800069FB134802686868131A2068401C002809
:1035900001D1002617E00F4928680968884204D045
:1035A0006868904201D801260DE02068984207D94A
:1035B0002068C01A20602846FFF7DCFB002602E0E6
:1035C000002020600126FFF753FB304670BD00004D
:1035D000180000202C000020FFB585B01746B80069
:1035E000FFF71CFA0646002E0BD05C20FFF716FAF8
:1035F0000446002C01D0266304E03046FFF74CFB64
:1036000000E00024002C10D000220F990E986B4689
:1036100013C303923A46089B06990598FFF795F85D
:103620002046FEF73FFF012501E00025ED43284637
:1036300009B0F0BD06490968002901D1012006E062
:1036400004490968002901D1022000E000207047E8
:10365000200000203C000020F8B5002000904248E7
:103660000068002872D141480068451C3F48056049
:10367000002D1CD13E4800680068002801D10120BF
:1036800000E00020002802D172B600BFFEE73848F3
:103690000768384800683649086036480760364889
:1036A0000068401C34490860FFF72CF900BF33481C
:1036B000006885423DD300BF2D480068006800289F
:1036C00001D1012000E00020002804D00020C043E8
:1036D0002A4908602CE026480068C068C46866680B
:1036E000B54202D22548066022E0201DFFF766FAA7
:1036F000A06A002803D020461830FFF75FFA20495F
:10370000E06A0968884202D91D49E06A086014220B
:10371000E16A51431B4A8818211DFFF78EFA1A49A6
:10372000E06A0968C96A8842C6D301200090C3E7ED
:1037300000BF15480068C06A142148431149085861
:10374000012801D90120009005E0FFE70F4800683B
:10375000401C0E4908600E480068002801D0012076
:1037600000900098F8BD00003C00002018000020E8
:10377000080000200C0000202C0000203400002055
:103780001C000020A40000200400002024000020D1
:103790002800002070B505462C460026002D35D0A7
:1037A0001B480068844201D1012000E0002000286D
:1037B00002D172B600BFFEE7206D002802D172B6BA
:1037C00000BFFEE7206D401E2065E16CE06A884284
:1037D0001CD0206D002819D1201DFFF7EFF9E06CF7
:1037E000E0620721E06A081AA0610A49E06A0968F4
:1037F000884202D90749E06A08601422E16A51430D
:10380000054A8818211DFFF718FA0126304670BDB9
:10381000040000201C000020A400002070B5054614
:103820002C460026002D42D02249E06A0968C96A68
:10383000884235D2A069C00FC007002805D11D48B5
:103840000068C06A0721081AA0611422E06A504388
:10385000194A80186169814201D1012000E00020ED
:10386000002817D0201DFFF7A9F912480068C06A88
:10387000E0621249E06A0968884202D90F49E06AA9
:1038800008601422E16A51430B4A8818211DFFF792
:10389000D4F903E007480068C06AE062012606E048
:1038A0000449E06C0968C96A884200D201263046A2
:1038B00070BD000004000020A40000201C000020B7
:1038C00070B50646F068C468002C02D172B600BF1D
:1038D000FEE720461830FFF771F915480068002808
:1038E00013D1201DFFF76AF91249E06A096888427E
:1038F00002D91049E06A08601422E16A51430E4A75
:103900008818211DFFF799F904E0214618310B486A
:10391000FFF793F90A49E06A0968C96A884204D93D
:10392000012501200749086000E00025284670BDF8
:103930003C0000201C000020A400002058010020B2
:10394000040000202800002070B500240026324822
:103950000068002802D172B600BFFEE7FFF77AF9CF
:103960002D480068401E2C49086008460068002861
:103970004DD12A480068002849D022E02848C06874
:10398000C46820461830FFF719F9201DFFF716F913
:103990002449E06A0968884202D92249E06A08603D
:1039A0001422E16A5143204A8818211DFFF745F986
:1039B0001E49E06A0968C96A884202D301201C498D
:1039C000086017480068002801D1012000E00020AD
:1039D0000028D3D0002C01D0FEF794FF15480568CD
:1039E000002D0DD000BFFFF737FE002802D00120C8
:1039F0000F4908606D1E002DF5D100200D490860AB
:103A00000B480068002802D00126FFF785F9FFF770
:103A10002FF9304670BD00003C000020140000204B
:103A2000580100201C000020A400002004000020F9
:103A3000280000202400002040BA7047C0BA704718
:103A40000138FDD170470000F7B50325AD06286A9F
:103A500082B016460C46400840002862286A0221BF
:103A600008432862286A8007FCD466206860012722
:103A70002F61A86AC005FCD5992068602F61A86AEB
:103A8000C005FCD5FF209130FFF7DAFFFF2301339B
:103A9000AB626846EF60352169602F61A96AC9058C
:103AA000FCD5AB62A969EF60C9B205226A602F61DB
:103AB000AA6AD205FCD5AB62AA690902D2B2114347
:103AC0000180C80702D0032005B0F0BDAB62686971
:103AD000FF210831884368616869C91E084368612D
:103AE00002980002483068600820A860EE602F61EC
:103AF000A86AC005FCD5FF200130A8620023F61C8F
:103B0000B0080ED0B2081148006899006054060A47
:103B100009194E70060C000E8E705B1CC8709A421C
:103B2000F1D8FF200130A8626869FF21083188437D
:103B30006861686938436861286A80088000286283
:103B4000286A38432862002005B0F0BD8000000CD0
:103B5000032080064169FF22083291434161426996
:103B600001210A434261026A920892000262026ADB
:103B70000A43026270470000002003218906096A97
:103B8000490849000322920611621146096A02227D
:103B9000114303229206116200BF03218906096ABC
:103BA000022211400229F8D0D1010322920691622B
:103BB0000321D1609F2151600121116100BF0321C8
:103BC0008906896AFF22013211409142F7D103220E
:103BD00092069162114688694969FF220832914331
:103BE00003229206516111464969012211430322C1
:103BF000920651611146096A8908890011621146CD
:103C0000096A0122114303229206116270470000E3
:103C10000000000001020304000001020100000096
:103C2000000000000200000000000000EC3C000169
:103C3000F43C000119090001C83C0001D03C00011E
:103C4000010B0001C43C00015C3C0001550A00016D
:103C5000C03C0001903C0001650900016C6F6720C9
:103C60005B6F6E7C6F66665D3A2061637469766532
:103C7000207072696E74696E672073776974636807
:103C8000202864656661756C74206F666629000083
:103C90006C6564203C317C323E203C6F6E7C6F66EC
:103CA000667C746F67676C653E3A20636F6E7472F2
:103CB0006F6C20626F617264204C4544000000000C
:103CC0006C6564006C6F670076657273696F6E0077
:103CD00073686F77206669726D776172652F636CA8
:103CE0006F636B20696E666F0000000068656C7022
:103CF000000000006C69737420616C6C20636F6D50
:103D00006D616E6473000000283D0001000000201A
:103D1000700000000A160001983D000170000020AC
:103D2000C82900001A1600010090D003000000000E
:103D30000000000000000000000000000000000083
:103D40000000000000000000000000000000000073
:103D50000000000000000000000000000000000063
:103D60000000000000000000AAAAAAAA00000000AB
:103D70000000000000000000000000000000000043
:103D80000000000000000000000000000000000033
:083D900000000000000000002B
:04000005010000C135
:00000001FF
